:100000000C94EE040C940B050C940B050C940B054E
:100010000C940B050C940B050C940B050C940B0520
:100020000C940B050C940B050C942E260C940027B5
:100030000C9477200C940B050C940B050C940B0579
:100040000C940B050C940B050C940B050C940B05F0
:100050000C940B050C94FF200C940B050C940B05D1
:100060000C940B050C940B050C940B050C940B05D0
:100070000C940B050C940B050C940B050C940B05C0
:100080000C940B050C940B050C940B050C940B05B0
:100090000C940B050C940B050C940B050C940B05A0
:1000A0000C940B050C940B050C940B05C608C608A4
:1000B000F208F2085A097809900A900A83091C0A82
:1000C0002D0A2D0A6D2794278C2894278C28E02749
:1000D00003288C285A286928000058006200000074
:1000E00059005A005B00630057005C005D0000008F
:1000F0005F00600061005E00530054005500560030
:100100003A003B003C003D0044454255473A2064DC
:10011000697361626C65642E0A0044454255473A32
:1001200020656E61626C65642E0A000A002530321B
:1001300058006C65645F7461736B3A20004F6E65A4
:1001400073686F743A206163746976653A20256438
:100150000A000A0025303862003A20002530325863
:10016000000A722F632030313233343536370A00BB
:10017000290A002575002F002575005D28002564DB
:100180000020002564002000256400200025640074
:100190007C0025303258006D6F7573656B65792072
:1001A0005B62746E7C782079207620685D287265A9
:1001B000702F61636C293A205B00313A0964656CE9
:1001C0006179282A31306D73293A2025750A323A2F
:1001D00009696E74657276616C286D73293A202501
:1001E000750A333A096D61785F73706565643A200A
:1001F00025750A343A0974696D655F746F5F6D61C6
:10020000783A2025750A353A09776865656C5F6D1F
:1002100061785F73706565643A2025750A363A091E
:10022000776865656C5F74696D655F746F5F6D613C
:10023000783A2025750A00703A097072696E742048
:1002400076616C7565730A643A0973657420646538
:100250006661756C74730A75703A092B310A646EA5
:100260003A092D310A6C743A092B31300A72743A0A
:10027000092D31300A4553432F713A09717569745C
:100280000A0A7370656564203D2064656C746120A2
:100290002A206D61785F7370656564202A2028725A
:1002A0006570656174202F2074696D655F746F5F80
:1002B0006D6178290A77686572652064656C746180
:1002C0003A20637572736F723D25642C20776865E0
:1002D000656C3D25640A53656520687474703A2F17
:1002E0002F656E2E77696B6970656469612E6F7218
:1002F000672F77696B692F4D6F7573655F6B6579D4
:10030000730A004D3E20004D25753A25733E2000AE
:100310003F0A003D2025750A003F0A0064656661BA
:10032000756C74730A0025750A003F0A000A092DCE
:100330002056616C756573202D0A00710A000A0948
:100340002D204D6F7573656B6579202D0A003F0078
:10035000433E20004C25640A000A092D2053746195
:10036000747573202D0A686F73745F6B6579626FA3
:100370006172645F6C65647328293A2025303258B5
:100380000A6B6579626F6172645F70726F746F631C
:100390006F6C3A20253032580A6B6579626F617252
:1003A000645F69646C653A20253032580A74696D5F
:1003B00065725F72656164333228293A20253038CE
:1003C0006C580A000A092D2056657273696F6E20F9
:1003D0002D0A5649443A2030784645454428536E04
:1003E000616D656C6C697429205049443A203078FD
:1003F0003030303028736E616D706164292056454D
:10040000523A203078303030310A4255494C443A23
:100410002020284665622032382032303232290AC4
:100420004F5054494F4E533A204C554641204D4F62
:100430005553454B45592045585452414B45592039
:10044000434F4E534F4C4520434F4D4D414E44205A
:10045000343039360A4743433A20352E342E302083
:100460004156522D4C4942433A20322E302E3020F4
:100470004156525F415243483A20617672350A0034
:100480000A092D20436F6E736F6C65202D0A45534A
:10049000432F713A09717569740A6D3A096D6F7568
:1004A00073656B65790A000A092D204D61676963E0
:1004B000202D0A443A094465627567204D657373BF
:1004C00061676520546F67676C650A583A094D612A
:1004D00074726978204465627567204D6F64652089
:1004E000546F67676C65202D2053686F77206B65AC
:1004F000797072657373657320696E206D617472B3
:10050000697820677269640A4B3A094B6579626FB2
:1005100061726420446562756720546F67676C651B
:10052000202D2053686F77206B6579707265737327
:10053000207265706F72740A4D3A0944656275677E
:10054000204D6F75736520546F67676C650A563A66
:100550000956657273696F6E0A533A095374617470
:1005600075730A433A09416374697661746520437F
:100570006F6E736F6C65204D6F64650A46312D4652
:1005800031303A0953776974636820746F204C6185
:1005900079657220302D392028463130203D204C9D
:1005A00030290A302D393A09537769746368207409
:1005B0006F204C6179657220302D390A47524156BF
:1005C000453A0953776974636820746F204C6179E8
:1005D000657220302028616C7465726E61746529C3
:1005E0000A423A094A756D7020746F20426F6F7429
:1005F0006C6F616465720A4553433A094A756D70C0
:1006000020746F20426F6F746C6F61646572202874
:10061000616C7465726E617465290A453A0950729D
:10062000696E7420454550524F4D2053657474696E
:100630006E67730A4253504143453A09436C656102
:100640007220454550524F4D0A006B65796D6170BF
:100650005F636F6E6669672E7261773A202530326C
:10066000580A2E737761705F636F6E74726F6C5F80
:10067000636170736C6F636B3A2025750A2E63613A
:1006800070736C6F636B5F746F5F636F6E74726FA8
:100690006C3A2025750A2E737761705F6C63746CF9
:1006A0005F6C6775693A2025750A2E737761705FF4
:1006B0007263746C5F726775693A2025750A2E73D0
:1006C0007761705F6C616C745F6C6775693A202547
:1006D000750A2E737761705F72616C745F726775F3
:1006E000693A2025750A2E6E6F5F6775693A202575
:1006F000750A2E737761705F67726176655F6573E7
:10070000633A2025750A2E737761705F6261636BAF
:10071000736C6173685F6261636B73706163653A88
:100720002025750A2E6E6B726F3A2025750A0064BB
:10073000656275675F636F6E6669672E7261773A8F
:1007400020253032580A2E656E61626C653A20258C
:10075000750A2E6D61747269783A2025750A2E6BC0
:100760006579626F6172643A2025750A2E6D6F7526
:1007700073653A2025750A006565636F6E66696763
:100780003A0A64656661756C745F6C617965723A8A
:100790002025750A003F000A6D6F7573653A206F5A
:1007A00066660A000A6D6F7573653A206F6E0A00FF
:1007B0000A6B6579626F6172643A206F66660A003F
:1007C0000A6B6579626F6172643A206F6E0A000A83
:1007D0006D61747269783A206F66660A000A6D610D
:1007E000747269783A206F6E0A000A6465627567F0
:1007F0003A206F66660A000A64656275673A206F80
:100800006E0A000A0A4A756D70696E6720746F205F
:10081000626F6F746C6F616465722E2E2E200043C0
:100820003E2000436C656172696E672045455052F9
:100830004F4D0A000A002530325820006B6579625E
:100840006F6172645F7265706F72743A20005B73DF
:100850005D005B575D005B535D005B525D005B4478
:100860005D005B435D00100373006E0061006D006E
:100870007000610064000000140353006E0061000A
:100880006D0065006C006C006900740000000403DA
:10089000090409025B00030100A0FA090400000139
:1008A0000301010009211101000122400007058117
:1008B00003080001090401000103000000092111DF
:1008C000010001227B0007058203200001090402C8
:1008D000000203000000092111010001222200078B
:1008E0000583032000010705030320000112010016
:1008F0000200000008EDFE000001000102000106F8
:1009000031FF0974A1010975150026FF00952075B6
:100910000881020976150026FF00952075089102CE
:10092000C005010902A10185020901A100050919FB
:1009300001290815002501950875018102050109A5
:100940003009311581257F95027508810609381512
:1009500081257F950175088106050C0A38021581ED
:10096000257F950175088106C0C005010980A10198
:10097000850319012AB700150126B70095017510E6
:100980008100C0050C0901A101850419012AA002FA
:10099000150126A002950175108100C00501090608
:1009A000A101050719E029E7150025019508750142
:1009B00081029501750881010507190029FF1500BD
:1009C00026FF00950675088100050819012905957F
:1009D0000575019102950175039101C011241FBE97
:1009E000CFEFDAE0DEBFCDBF11E0A0E0B1E0E4E997
:1009F000F2E502C005900D92A23FB107D9F722E0BF
:100A0000A2EFB1E001C01D92A93BB207E1F70E943D
:100A1000CF160C9448290C940000FF93EF93E091BB
:100A2000F201F091F301309709F00995EF91FF91F0
:100A30000895FC018591803011F0EFDFFBCF089520
:100A4000FF27E0E230E247FF0CC0419597FF09C065
:100A5000EDE26095709580959095611D711D811DE9
:100A6000911D27FF02C0219530E350E2AA27660FAF
:100A7000771F881F991FAA1FA41710F0A41B639546
:100A80005A95A9F7AA3008F0A95FA05DAF93F39536
:100A9000611571058105910541F7ED3211F4EF9370
:100AA000F395F21718F43F93F395FBCF8F91B5DFD1
:100AB000FA95E1F70895E991F9918591803021F057
:100AC000853219F0AADFF9CF089520E0E894559116
:100AD0005532C1F3503311F4689455915A3348F4A8
:100AE000505390F3220F022E220F220F200D250FBC
:100AF000F4CF0EF4219589919991533619F3533718
:100B000029F1533559F1BC0188279927E8945C36BF
:100B100021F48991999168945591543639F446EFAE
:100B20007EF077FF0DC08FEF9FEF0AC055374AE088
:100B300039F0583540E121F0523642E009F008958D
:100B4000FF93EF937DDFEF91FF91B7CFFF93EF938B
:100B5000FC0181918030B9F360DFFBCFFF93EF930D
:100B600068DFF1CFDF93CF93CDB7DEB72596A3DF54
:100B7000CF91DF91089581E0089581E008950C946C
:100B8000BD0508950C94C1051F93CF93DF9300D04A
:100B900000D01F92CDB7DEB749835A836B83309163
:100BA000F50189819A81311114C0662359F02223FD
:100BB00049F00E94CB0C182F682F89819A810E94DE
:100BC000760C03C00E94A00C182F69817A81812FB6
:100BD00004C00E94CB0C69817A810F900F900F9016
:100BE0000F900F90DF91CF911F910C940014FC0196
:100BF000262F408151816281738184810C94C405C8
:100C000081E00895CF93DF93EC0160E00E94F70547
:100C1000BE01DF91CF910C94C2050C9487150C9402
:100C2000831508950E94200B0E9411062FEF84E384
:100C30009CE0215080409040E1F700C000000C94FF
:100C400025210F931F93CF93DF938C0161E00E94C6
:100C5000F705EC01B8010E94BF05882309F45BC0C9
:100C6000B801CE010E94051F882309F454C0B801C1
:100C7000CE010E94E719882309F44DC0B801CE01C6
:100C80000E94611E882309F446C0F80182818823EE
:100C9000D9F1CF3D8CE5D80779F140F4C115FCE5D9
:100CA000DF0791F0C130DC4591F02EC0CC35EDE589
:100CB000DE0741F1CD35FDE5DF0709F1CB35DD4537
:100CC00019F50E94621120C00E94120624C0809172
:100CD0006702C82FC095C170C0FB80F9809367027E
:100CE000CC2329F08AE191E00E94190514C088E024
:100CF00091E00E94190510C00E9416120CC00E94BB
:100D0000591102C00E946511C801DF91CF911F9156
:100D10000F910C94BB05C0E08C2FDF91CF911F91F8
:100D20000F9108950E945A200C94BD060E94C0069F
:100D30000C9460208295982F937344E0949F9001C7
:100D400011248C7C86958695282B822F8575880F9B
:100D50002A7A2695822B089508950C94AC0681E09A
:100D600008950C94AF060895CF93C82F0E94AD0646
:100D70008C2F0E94B106CF91089580E00C94B406A8
:100D80000E94611F0C94B406CF930E94611FC82F6C
:100D90008091F401C81741F1C093F401809167027A
:100DA00082FF1EC080FF04C082E391E00E9419050B
:100DB0008091670280FF0CC01F92CF938DE291E07B
:100DC0009F938F930E94B2050F900F900F900F90FA
:100DD0008091670280FF04C08BE291E00E941905B8
:100DE0008C2FCF910C94B406CF910895CF93DF93BD
:100DF000CDB7DEB72B970FB6F894DEBF0FBECDBFD1
:100E00004F83588769877A878B8761110E94911079
:100E10009E012F5F3F4F86E0F90111928A95E9F715
:100E200085E0FE013796D90101900D928A95E1F790
:100E300089819A814C815D81452B31F09F3F31F44E
:100E400091E08F3F19F403C091E001C090E090FF62
:100E500009C049815A816B817C818D819E810E946C
:100E6000B20F05C0C9010E9400068111F2CF2B9676
:100E70000FB6F894DEBF0FBECDBFDF91CF910895BE
:100E8000FC01808191810E940D0D0895CF938823EC
:100E900009F4A9C0C82F8238C1F40E94611F81FDE6
:100EA000A2C069E380910201909103010E94322067
:100EB0000E94B3102FEF81EE94E0215080409040CB
:100EC000E1F700C0000069E319C0833801F50E9412
:100ED000611F80FD88C063E580910201909103014C
:100EE0000E9432200E94B3102FEF81EE94E0215037
:100EF00080409040E1F700C0000063E5809102016E
:100F0000909103010E943420CF910C94B310843847
:100F1000C1F40E94611F82FD66C067E480910201F6
:100F2000909103010E9432200E94B3102FEF81EEB6
:100F300094E0215080409040E1F700C0000067E459
:100F4000DDCF8CEF8C0F813AF8F48C2F0E940A1EB3
:100F5000811149C06C2F80910201909103010E9480
:100F6000FC1F882349F06C2F8091020190910301AE
:100F70000E9434200E94B3106C2F80910201909146
:100F800003010E943220C0CF80E28C0F883048F4E9
:100F9000C77081E001C0880FCA95EAF70E947410FB
:100FA000B3CFEBE5EC0FE33040F4F0E0E95BFE4F4C
:100FB000808190E0CF910C94C41FE8E5EC0FE731FD
:100FC00050F4F0E0EE0FFF1FE75EFE4F808191814D
:100FD000CF910C94DA1FCD3E30F08C2F0E94541725
:100FE000CF910C942618CF910895882309F464C0FA
:100FF000823879F40E94611F81FF5EC069E38091AD
:101000000201909103010E9432200E94B31069E313
:1010100010C08338B1F40E94611F80FF4DC063E5AA
:1010200080910201909103010E9432200E94B3102E
:1010300063E580910201909103010E9434200C9499
:10104000B310843879F40E94611F82FF35C067E4D1
:1010500080910201909103010E9432200E94B310FE
:1010600067E4E7CF9CEF980F913A10F4682FE1CF37
:1010700090E2980F983050F4877091E001C0990F7A
:101080008A95EAF7892F0E947A10D9CF9BE5980FAD
:10109000933020F480E090E00C94C41F98E5980F02
:1010A000973120F480E090E00C94DA1F8D3E20F020
:1010B0000E94AF170C94261808951F93CF93DF93C7
:1010C000182FEB010E944607209741F08FE99FE01F
:1010D0000197F1F700C000002197F6CF812FDF9133
:1010E000CF911F910C94F507893319F060E070E0FF
:1010F00002C060E570E00C945D08882321F00E9436
:1011000074100C94B3100895882321F00E947A1073
:101110000C94B3100895CF92DF92EF92FF920F9349
:101120001F93CF93DF937C01D62FC72FFC01128131
:10113000058102950F700E946A108823B9F011236F
:10114000A9F08C2F807F803421F080E28D0F8830D1
:1011500068F080919B0282FD09C082E00E94131119
:101160000E946A1091E0D82ED92601C0D12CCC2E35
:10117000C2948FE0C8228C2D90E08C30910508F04D
:10118000CFC1FC01EA5AFF4F0C94DF288C2F807FDF
:10119000CF70882311F0C295C07F112399F0CC2322
:1011A00009F4AAC180E28D0F883010F0D11104C07B
:1011B0008C2F0E94741003C08C2F0E9484100E94F8
:1011C000B3109AC18D2F0E94F507CC2309F4A8C152
:1011D00080E28D0F883038F1DD2329F18C2F0E94B9
:1011E0008A1024C08C2F807FCF70803211F0C2957E
:1011F000C07FDD2319F0D130A1F13DC080919B0269
:1012000082FF17C0112349F0CC2329F08C2F0E94B4
:1012100074100E94B31080E070C180E00E94F50756
:10122000CC2309F47DC18C2F0E947A100E94B31048
:1012300077C1112371F0002341F0013031F40E9495
:1012400094108C2B0E949C106BC10E9494108C2BCC
:101250001DC0002319F0013009F462C10E94A910D9
:1012600025C0112321F0063008F05AC10EC0053008
:1012700008F056C11BC0112361F0002331F0F701C3
:10128000858180FF39C18F7085838C2F0E947D08F6
:1012900047C1002359F0D93309F03FC1FFEF07EEF2
:1012A00013E0F15000401040E1F735C18C2F0E944F
:1012B000840836C18C2F86958695837019F081300D
:1012C00061F02EC1112321F08D2F9C2F937002C04D
:1012D00080E090E00E94C41F2BC1112321F08D2FCC
:1012E0009C2F937002C080E090E00E94DA1F20C122
:1012F0008D2F112319F00E94541702C00E94AF17BE
:101300000E94261815C18C2F837009F047C0111157
:101310000BC12D2F229526952770220F220F6D2F9E
:101320006F70862F90E0A0E0B0E0022E04C0880F1E
:10133000991FAA1FBB1F0A94D2F7D4FF10C04FE019
:1013400050E060E070E004C0440F551F661F771F37
:101350002A95D2F7409550956095709503C040E06E
:1013600050E0BA01C695C695C3708A019B01082B4F
:10137000192B2A2B3B2BC901B801C23049F058F474
:10138000C13019F00E948C0BCFC00E947A0BCCC0E8
:101390000E949E0BC9C00E94780BC6C0112319F091
:1013A0008C2F817001C08695882309F4BDC02D2F34
:1013B000229526952770220F220F6D2F6F70862F92
:1013C00090E0A0E0B0E0022E04C0880F991FAA1F91
:1013D000BB1F0A94D2F7D4FF10C04FE050E060E08A
:1013E00070E004C0440F551F661F771F2A95D2F77F
:1013F000409550956095709503C040E050E0BA016B
:10140000C695C695C3708A019B01082B192B2A2B00
:101410003B2BC901B801C23049F058F4C13019F072
:101420000E94510C81C00E943F0C7EC00E94630C40
:101430007BC00E94B20B78C0CF70112339F08C2F83
:101440000E94D80B8D2F0E947D086EC08D2F0E94A8
:1014500084088C2F0E94F90B67C0D23F21F128F439
:10146000D03F41F0D13FC1F043C0D33F19F1D43F49
:1014700079F03EC0112341F0053008F051C08C2FA7
:101480008F710E941E0C4CC0063008F049C0F7CF87
:1014900080919B0282FF18C0112339F08C2F8F712D
:1014A0000E94D80B3DC01123C9F38C2F8F710E946D
:1014B000F90B36C0112329F08C2F8F710E94C30BBA
:1014C0002FC00E94BE0B2CC0112349F0CF718C2F6E
:1014D0000E94D80B63E08C2F0E94F81021C081E09D
:1014E0000E9413110230E0F082E00E94131118C034
:1014F000112331F0002391F28D2F0E94460710C076
:10150000002399F2D93349F41FEF27EE33E011504D
:1015100020403040E1F700C000008D2F0E94F50709
:1015200088EF8C0D843020F40E94611F0E94B40665
:10153000DD20C9F00E94661080FD15C0F7011282FF
:101540000E9460100E94D80BC7010E94D40A0E941A
:101550006010DF91CF911F910F91FF90EF90DF907E
:10156000CF900C94F90BDF91CF911F910F91FF90C9
:10157000EF90DF90CF9008950F931F93CF93DF9359
:10158000EC01688179818A810E94180D8C010E948A
:10159000750C0E94660BB801CE010E948B08DF918A
:1015A000CF911F910F910895CF93DF93EC01988114
:1015B00089812B813C81232B31F08F3F31F481E0F5
:1015C0009F3F19F403C081E001C080E080FD1DC091
:1015D000CE010E942106811110C00E946A1088234A
:1015E000A1F08A81882389F080919B0282FD0DC041
:1015F00082E0DF91CF910C941311CE010E94BC0ABE
:10160000CE01DF91CF910C940206DF91CF91089526
:1016100080E090E00E94C41F80E090E00E94DA1F0A
:101620000E9491100E94B3100E94D9190C942618A0
:1016300080910201909103010E9436200C94080BC6
:101640000E9481100C94180B92959F70963079F03F
:1016500010F4925001C09A50923068F4803F69F0C3
:1016600018F4883E40F409C0843F29F406C0883E3F
:1016700020F0813F11F080E0089581E00895FC01A1
:10168000808191810E940D0D0E94240B0895CF93BB
:10169000DF9300D000D01F92CDB7DEB70F900F9030
:1016A0000F900F900F90DF91CF910895CF93DF931C
:1016B00000D000D000D0CDB7DEB726960FB6F89494
:1016C000DEBF0FBECDBFDF91CF910895089508957D
:1016D0000C94670B0C94680B0E946A0B60930902D0
:1016E00070930A0280930B0290930C020C94080BE7
:1016F0000C946C0B0F931F930091090210910A0236
:1017000020910B0230910C02602B712B822B932BBA
:101710001F910F910C946C0B0F931F930091090272
:1017200010910A0220910B0230910C026023712368
:10173000822393231F910F910C946C0B0F931F9393
:101740000091090210910A0220910B0230910C02C3
:1017500060277127822793271F910F910C946C0BA0
:101760000C94670B0E94B00B609305027093060205
:1017700080930702909308020C94080B60E070E0DD
:10178000CB010C94B20B0F931F9341E050E060E04B
:1017900070E08A019B0104C0000F111F221F331F3C
:1017A0008A95D2F7C901B8011F910F910C94B20B21
:1017B0000F931F9341E050E060E070E004C0440FDD
:1017C000551F661F771F8A95D2F780910502909169
:1017D0000602A0910702B09108028A019B01082B22
:1017E000192B2A2B3B2BC901B8011F910F910C9487
:1017F000B20B0F931F9341E050E060E070E004C033
:10180000440F551F661F771F8A95D2F74095509554
:10181000609570958091050290910602A091070253
:10182000B09108028A019B01082319232A233B2334
:10183000C901B8011F910F910C94B20B0F931F9324
:1018400041E050E060E070E004C0440F551F661FA7
:10185000771F8A95D2F78091050290910602A09198
:101860000702B09108028A019B01082719272A273D
:101870003B27C901B8011F910F910C94B20B0F9334
:101880001F930091050210910602209107023091EA
:101890000802602B712B822B932B1F910F910C94BC
:1018A000B20B0F931F930091050210910602209135
:1018B00007023091080260237123822393231F9132
:1018C0000F910C94B20B0F931F930091050210918E
:1018D00006022091070230910802602771278227B3
:1018E00093271F910F910C94B20B0895990F990FA4
:1018F000890FE82FE695E695E695877051E001C0DF
:10190000550F8A95EAF785E0E89FF0011124EA5027
:10191000FE4F20E030E070E04081CB01022E02C09B
:10192000969587950A94E2F781708195842785239F
:10193000842781932F5F3F4F2530310569F7089544
:10194000990F990F890F682F669566956695982F60
:10195000977085E0689FB001112440E050E080E07E
:10196000FB01E40FF51FEA50FE4F208130E0092E05
:1019700002C0369527950A94E2F721703327042E8A
:1019800001C0220F0A94EAF7822B4F5F5F4F453068
:10199000510531F70895BF92CF92DF92EF92FF92F7
:1019A0000F931F93CF93DF938C01C0900502D090CB
:1019B0000602E0900702F0900802809109029091DF
:1019C0000A02A0910B02B0910C02C82AD92AEA2A75
:1019D000FB2ACFE1D0E0D701C6010C2E04C0B6959A
:1019E000A795979587950A94D2F780FD04C0219713
:1019F00090F7B12C07C0BC2EB8018C2F0E94141494
:101A00000197A9F38B2DDF91CF911F910F91FF903B
:101A1000EF90DF90CF90BF900895CF93DF93EC01CC
:101A20000E94CB0CBE010E941414DF91CF91089547
:101A30001F93CF93DF93EB019091F501992321F050
:101A4000CB010E940D0D13C0882349F0CB010E94E9
:101A5000CB0C182F682FCE010E94760C04C0CB014E
:101A60000E94A00C182FBE01812F0E941414DF9138
:101A7000CF911F9108951F93CF93DF93C0910D02D3
:101A800016E080910E02C81799F0D0E01C9FF0017B
:101A90001D9FF00D1124E15FFD4F40815181628156
:101AA0007381848195810E94560B2196C770E9CF7E
:101AB000DF91CF911F91089540913F0250914002D4
:101AC00060914102709142028091430290914402E0
:101AD0000C94560BEF92FF920F931F93CF93DF93CB
:101AE0008091440282958F7009F065C08091410217
:101AF000882309F460C080910D02F0900E021091CD
:101B00003F0200914002609142027091430291E0D5
:101B10001F3F09F090E0C0910001D0910101292FF1
:101B200096E0E92E8F1509F446C06115710521F084
:101B30000F3F21F030E003C031E001C0322F90E0D0
:101B400030FD36C0E89EF001E99EF00D1124DF0162
:101B5000A15FBD4F11963C911197301329C03C9164
:101B6000311326C012963C911297311121C0139661
:101B70004D915C911497461B570B4C175D07C0F4B1
:101B8000809144028F70806180934402EC5EFD4F2F
:101B900080818F70806180838FE392E00E94D40AFD
:101BA000DF91CF911F910F91FF90EF900C943B0D1F
:101BB00001968770B7CFDF91CF911F910F91FF9062
:101BC000EF9008959F92AF92BF92CF92DF92EF92E3
:101BD000FF920F931F93CF93DF93CDB7DEB761973B
:101BE0000FB6F894DEBF0FBECDBF8C0185E0F801C3
:101BF000DE011D9601900D928A95E1F7D8011296AB
:101C0000EC9090913F02E09140022091420230918D
:101C100043022115310531F0EF3F31F481E09F3F60
:101C200019F403C081E001C080E0B82FB1709B2E91
:101C300080FD47C1D8014C9111965C911197139684
:101C4000AD90BC9014978FE3C82E82E0D82EF09010
:101C50004102B501621B730B20910001309101011B
:101C6000FF2009F4D9C0809144026217730708F07D
:101C700095C0282F207F09F052C05E1313C049136E
:101C800011C0FE2CE1100EC08F7080618093440261
:101C90000E945C0DC6010E94D40A80914402F801A2
:101CA00085834DC1AB2831F05F3F31F481E04F3F78
:101CB00019F403C081E001C080E080FD03C081E031
:101CC0008E2502C080E090E0F82FF170FF2E80FF9B
:101CD0001CC080910D0220910E0236E0821709F49B
:101CE0000BC190E0389FF001399FF00D1124E15FA6
:101CF000FD4F6181561306C06081461303C06281A7
:101D0000E61203C001968770E9CFFE2CEE2009F49D
:101D100016C18091440281608093440254C05E13D6
:101D200006C0491304C0E11002C0F80199C0C801FF
:101D30000E943F0B882361F1EE2051F12091440273
:101D4000822F82958F7090E0029774F080913F020D
:101D50009091400298878F831986BB86AA862C872C
:101D6000CE0107960E94D40A86E0F801AFE3B2E004
:101D700001900D928A95E1F70E946A0D0E945C0D18
:101D80000AC05E1711F1C8010E943F0B81112CC0DF
:101D9000C8010E94D40AFF24F394D1C0282F207FC9
:101DA00081F77A2DB98AA88A6E2D89890E94470BFE
:101DB0008FE392E00E94D40A86E0D6011D928A95B4
:101DC000E9F70E945C0DF12CBAC04913DCCFE11099
:101DD000DACFF8018583C8010E94D40A86E0D601D3
:101DE0001D928A95E9F7ABC0EE2091F22091440252
:101DF000822F82958F7090E002970CF4B5CF80917E
:101E00003F02909140029A8389831B82BD82AC82FB
:101E10002E83CE010196A6CF6217730708F044C047
:101E2000FE2CEE2009F4B4CF5E1330C049132EC04F
:101E30002091440220FD21C0822F82958F70482F6F
:101E400050E041155105C9F0F80125834F30510587
:101E500041F08F5F982F9295907F822F8F70892B02
:101E60008583C8010E94D40A86E0F801AFE3B2E09E
:101E700001900D928A95E1F73CC086E0F801AFE34E
:101E8000B2E001900D928A95E1F759C0C8010E9415
:101E90003F0B811169CF809144028160809344029D
:101EA000C8010E94D40A4BC07A2DB98AA88A6E2D27
:101EB00089890E94470B86E0D6011D928A95E9F731
:101EC00018C0EE2009F464CFC8010E943F0BF82E21
:101ED000882309F45DCF86E0F801AFE3B2E001901A
:101EE0000D928A95E1F78FE392E00E9440070E94ED
:101EF0006A0D0E945C0D23C04D875E878D859E858F
:101F00000E940D0D292F22952F70223028F49F70EA
:101F100039F0811105C00BC0243028F49F7049F4BA
:101F2000805E883020F0C8010E94D40A9F2CF92CD2
:101F300006C0D80115969C91907F91F7F8CF8F2D10
:101F400061960FB6F894DEBF0FBECDBFDF91CF9183
:101F50001F910F91FF90EF90DF90CF90BF90AF90C7
:101F60009F9008951F93CF93DF93CDB7DEB72C9743
:101F70000FB6F894DEBF0FBECDBF4F835887698779
:101F80007A878B879C87CE0107960E94E20D882373
:101F9000D1F09F8188852A853B85232B31F08F3FA7
:101FA00031F481E09F3F19F403C081E001C080E07B
:101FB00080FD47C04F81588569857A858B859C85D2
:101FC0000E94560B3EC086E0FE013796DE01119658
:101FD00001900D928A95E1F7FF81E8856A857B85FE
:101FE0006115710531F0EF3F31F481E0FF3F19F4E5
:101FF00003C081E001C080E080FD23C020910E027B
:1020000030E0C90101968770992740910D0250E098
:1020100084179507F1F1F983EA837D836C8396E059
:10202000929FD001939FB00D1124A15FBD4FFE017F
:10203000319601900D929A95E1F780930E020E94DD
:102040003B0D16E080910D0290910E02891771F1FF
:10205000189FC0011124815F9D4F0E94E20D8823CB
:1020600029F1E0910D021E9FF0011124E15FFD4F67
:102070004081518162817381848195810E94560BD8
:1020800080910D0290E001968770992780930D0250
:10209000D9CF0E94200B10920E0210920D02EFE396
:1020A000F2E086E0DF011D928A95E9F72C960FB6E3
:1020B000F894DEBF0FBECDBFDF91CF911F91089581
:1020C00080914D02859585958595089580914D0265
:1020D0008770089590914D02977081E009F480E037
:1020E000089580915802089590915802892B809309
:1020F0005802089580959091580289238093580240
:10210000089510925802089590915702892B809358
:102110005702089580959091570289238093570222
:10212000089510925702089580914E0208950895DF
:102130000C9497100C94981090919B0292FD08C0FB
:1021400090914E02981721F080934E020C949A10B1
:10215000089580914E02882329F010924E0280E06B
:102160000C949A100895CF93DF93E0910201F091BF
:102170000301809158028083E0910201F0910301F4
:10218000908180915702892B808380914E02882311
:1021900081F0E0910201F09103019081892B80830D
:1021A00080910201909103010E94F01F81110E9411
:1021B000A910C0910201D091030148E050E065E40C
:1021C00072E0CE010E94F928892B69F088E0FE01B7
:1021D000A5E4B2E001900D928A95E1F7CE01DF917E
:1021E000CF910C946D1FDF91CF9108950C949710AF
:1021F00090919B0292FD10C098E0899F900111245C
:10220000262B20934D020E94D80B80914D0285957C
:10221000859585950C94F6100C94D80B10924D0270
:1022200080E00C94F61020914D02809582238093DB
:102230004D02982F977099F430E0482F082E000C2B
:10224000550B2417350759F090919B0292FD07C05A
:102250008595859585950E94F90B0C940E1108952E
:10226000CF9390919B0292FB222720F92817F9F037
:10227000C82F892FC0FB82F980939B0280919A021C
:1022800090919B020E94921182E00E941311809112
:10229000670280FF0CC01F92CF938DE391E09F9364
:1022A0008F930E94B2050F900F900F900F90CF91D7
:1022B000089580919B0282FB882780F991E089270D
:1022C0000C94301181E00C94301180E00C943011AA
:1022D0006FEF7FEF80E090E00C94322980E090E097
:1022E0000E940E2921E0893E9E4F09F020E0822FB6
:1022F000089582E090E00C94062983E090E00C942D
:102300000629CF9384E090E00E940629C82F82E23C
:1023100090E00E9406292C2F30E0A901582BCA0119
:10232000CF910895CF93C92F682F84E090E00E9449
:1023300014296C2F82E290E0CF910C941429AB0108
:10234000BC018FE090E00C942629AB01BC0183E135
:1023500090E00C94262960E070E0CB010C94A5116C
:1023600060E070E0CB010E949F110C94AB1169EE0C
:102370007EEF80E090E00E94322960E082E090E011
:102380000E94142960E083E090E00E9414291092DA
:10239000090210920A0210920B0210920C0260E0E5
:1023A00084E090E00E94142960E082E290E00E94C4
:1023B000142960E085E090E00E94142960E086E046
:1023C00090E00E9414296FEF87E090E00E941429AA
:1023D00040E050E0BA0188E090E00E94262960E0E9
:1023E0008DE090E00E94142940E050E0BA0188E1BD
:1023F00090E00E94262960E087E190E00E94142985
:1024000040E050E0BA018CE190E00E94262960E0B3
:1024100070E080E290E00E94322940E050E0BA0192
:1024200088E190E00E9426290C94B0110C94B71119
:10243000682F8EE090E00C9414290E94E4206093B1
:1024400063027093640280936502909366026093C6
:102450005F0270936002809361029093620208951C
:1024600085B7806885BF85B7806885BF089581E09E
:1024700008950C94371208950C943B120C943B125F
:102480000C943E120C943B120C9442120C943B128E
:102490000E94301289E093E20E94571F0E94461268
:1024A0000C9444120E943C120C943B120E9408159A
:1024B0000C94B3060E94CF200E9429160E94561247
:1024C0000C9440128F929F92AF92BF92CF92DF9264
:1024D000EF92FF920F931F93CF93DF93CDB7DEB7A9
:1024E0002A970FB6F894DEBF0FBECDBF0E943E16EE
:1024F000982E81110E941D1289E5A82E82E0B82E27
:1025000000E010E0802E802F0E942C15D82EF501BF
:10251000C1905F01C826B1F40F5F1F4F063011054F
:1025200089F78FEF89838A831B820E94D82081607C
:10253000782F9D838C8349815A816B818D810E9484
:10254000F6062FC08091670281FD0E943215E12CB2
:10255000FF24F3948C2D8F21F1F00E9439128823EF
:1025600099F0EE828F82DF2081E009F480E0888795
:102570000E94D8208160782F9A8789874E815F8159
:1025800068858A850E94F606F801E75AFD4F80812A
:10259000F826F08206C0E394FF0CF4E0EF12DACFE5
:1025A000BBCF81E0911001C080E02A960FB6F8946D
:1025B000DEBF0FBECDBFDF91CF911F910F91FF9076
:1025C000EF90DF90CF90BF90AF909F908F90089545
:1025D0000E9462120E94C6180C94C406CF93DF9327
:1025E0000E941914EC01811521E5920708F045C0FD
:1025F000811530E5930708F094C0883E910528F5D1
:10260000803E910508F0F8C0883A910570F4853A4B
:10261000910508F07CC08130910509F475C008F47B
:10262000E8C0049708F0E8C0E4C08F3B910508F0CB
:10263000E0C0C85AD0E0CC0FDD1FC65BDE4F09906A
:10264000D881C02DCE019464D8C0811540E2940792
:1026500058F4811551E0950708F0CEC08D3E9105E4
:1026600008F4C7C09065C9C0C11580E4D80708F454
:10267000C0C0DF70CE01906AC0C0811525E5920709
:10268000A8F4811534E5930708F095C0811543E55A
:10269000940708F07BC0811552E5950708F061C0EA
:1026A000D82FCC27CE01816F906AA7C0C11589E5CC
:1026B000D807A0F4C11528E5D20708F082C0C115DB
:1026C00036E5D30708F095C08C2F0E94AD148F71AA
:1026D00090E0D82FCC27CE0190628FC0C1154AE57B
:1026E000D40708F474C0CE0190568115904208F0CA
:1026F00080C08D2F8F710E94AD14DD27D0628F7145
:10270000AE01582BCA0179C081E090E076C0C55A6D
:10271000D0E0C858DE4F8881C82FD0E0CE01906449
:102720006CC074E0969587957A95E1F7282F237011
:102730003C2F337081E090E002C0880F991F3A95DA
:10274000E2F79C68AC01522B9A019C2F9F709695E2
:10275000969550E2959FE0011124C9018C2B9D2B89
:102760004CC08370992721E030E002C0220F331F54
:102770008A95E2F79C2F9695969580E2989FE001C6
:102780001124C22BD32BCE019C6837C083709927AC
:1027900021E030E002C0220F331F8A95E2F79C2F20
:1027A0009695969540E2949FE0011124C22BD32B7D
:1027B000CE019A6822C0D82FCC27CE01846F906AB0
:1027C0001CC0DC2FCC27CE01806F906A16C08C2FE6
:1027D0008F700E94AD1494E0D695C7959A95E1F755
:1027E000CF70D0E0DC2FCC27D0699E01282BC90107
:1027F00004C080E090E001C0CE01DF91CF91089548
:10280000E72FF0E096E0899FE00DF11D1124EE0F17
:10281000FF1FEE0FFF1FE60FF11DEE0FFF1FE85227
:10282000FF4F8591949108950E9400140E94EE122A
:1028300008958238910569F1B0F48133910509F466
:102840006DC048F48932910509F463C08A3291055C
:1028500009F469C008958533910509F455C0893399
:102860009105B9F00895833E910569F138F4803EF1
:102870009105B1F0823E910509F10895863E9105DA
:10288000A9F1873E9105B9F1843E910509F064C034
:1028900023C020919A0220FD4FC021FD4DC0089514
:1028A00080919A0280FD44C080919B0280FF44C0C9
:1028B00080919A0284FD42C083EE4DC080919A02BD
:1028C00082FF38C0F5CF80919A0282FD33C080919B
:1028D0009B0280FD31C0ECCF80919B0281FF32C012
:1028E00080919A0284FD2AC087EE35C080919A02B9
:1028F00083FF26C0F5CF80919A0283FD21C080918D
:102900009B0281FD1FC0ECCF80919A0285FD1CC007
:102910001DC080919A0285FD19C016C080919A024F
:1029200086FD16C017C080919A0286FD13C010C0A4
:1029300089E311C082EE0FC080EE0DC080E00BC0B5
:1029400086EE09C084EE07C089E205C085E303C0B6
:102950008AE201C081E390E0089590919A0292FF8B
:102960000DC0282F2871283019F4877F846006C095
:10297000282F2471243011F48B7F886093FF0DC0C1
:10298000282F2871283119F4877E846106C0282FEA
:102990002471243111F48B7E886120919B0220FFE9
:1029A0000DC0382F3871383019F4877F816006C028
:1029B000382F3171313011F48E7F886021FF0DC0C6
:1029C000282F2871283119F4877E816106C0282FAD
:1029D0002171213111F48E7E886194FD877E0895E6
:1029E0000C9468110E943E168FE39CE90197F1F761
:1029F00000C000000E943E1680E00E942C1580FF5F
:102A000004C00E94F0140C94252108950C94F21433
:102A10000E946E11811102C00E9416120E9479114B
:102A2000809367020E94811190939B0280939A0287
:102A30000E9406150E947D11682F70E080E090E0F2
:102A40000E94780B60910502709106028091070246
:102A5000909108020C94B00BE82FF0E0EE55FD4F7A
:102A600080810895CF92DF92EF92FF920F931F9390
:102A7000CF93DF9381E691E00E94190582EAE82E68
:102A800082E0F82EC0E0D0E09CE5C92E91E0D92E7E
:102A900004E511E0DF93CF93DF92CF920E94B2055D
:102AA00089E591E00E941905F70181917F010E945B
:102AB0009A061F928F931F930F930E94B20582E58F
:102AC00091E00E94190521968DB79EB708960FB622
:102AD000F8949EBF0FBE8DBFC630D105D9F6DF91E9
:102AE000CF911F910F91FF90EF90DF90CF900895BD
:102AF00080EA8A95F1F7089500C008950C9478153E
:102B000008950C9480150C9481150C9480150C94E8
:102B10008515F894E82FE295EF70F0E031A1282FA9
:102B20002F7081E090E001C0880F2A95EAF7982F76
:102B30009095932391A392A1892B82A378940895D1
:102B40000F931F93CF93DF93CBE7D1E089918F3F12
:102B500011F00E94891581E0CF37D807B9F7CFE788
:102B6000D1E005E811E089918F3F11F00E948915AD
:102B70000C171D07C1F7DF91CF911F910F91089599
:102B8000EF92FF920F931F93CF93DF93C62FD0E066
:102B9000C558DE4F28812F3F09F454C0042F162F4B
:102BA0007C01F894E22FE295EF70F0E081A1422FD2
:102BB0004F7021E030E001C0220F4A95EAF7822BE6
:102BC00081A382A12095282322A378940E947C15BA
:102BD0006FE771E0F701A7014A5F5F4FF12C302FDB
:102BE0003095DB012D91BD012F3FB1F0822F8295F1
:102BF0008F7090E0DC0190968C9190E02F7002C075
:102C0000959587952A95E2F780FD06C08081802BF7
:102C10008083FF24F39403C08081832380833196D3
:102C2000E417F507F1F688818F3F11F00E948915AE
:102C30006F2D812FDF91CF911F910F91FF90EF901A
:102C40000C947E15DF91CF911F910F91FF90EF9023
:102C500008950E94A01586E0E2EAF2E0DF01982FD5
:102C60001D929A95E9F7ECE9F2E0DF011D928A9551
:102C7000E9F786E00E948C160C940D06EF92FF9205
:102C80000F931F93CF93DF9300D000D000D0CDB728
:102C9000DEB78E010F5F1F4F86E0F80111928A9513
:102CA000E9F7F12CEE24E3944E2D6F2DC8010E941C
:102CB000C015F394EE0CF4E0FF12F6CF46E050E0BE
:102CC000B8018CE992E00E94F928FF24F394009760
:102CD00009F4F12C892B41F086E0F801ACE9B2E06F
:102CE00001900D928A95E1F72F2D46E062EA72E09D
:102CF0008CE992E00E948D160E940F068F2D269679
:102D00000FB6F894DEBF0FBECDBFDF91CF911F91FC
:102D10000F91FF90EF9008950895FF920F931F93E6
:102D2000CF93DF938C01F62ED72FC42F222349F0A7
:102D300081E080936A020E94D82090936902809378
:102D4000680280916A028823C1F0809168029091A4
:102D500069020E94F020059780F0EF2DFD2FD80129
:102D60004C2F50E0CD01801B910B841795071CF46C
:102D70008D918193F7CF10926A02DF91CF911F91CD
:102D80000F91FF9008950E9485230E945A120C947F
:102D900091230E9495230E94E8120C94B3230E9471
:102DA00076200E946C230E9448120E94C3160E9443
:102DB000C9160E945212FBCF8091710280FF06C09B
:102DC0006091090170E0660F771F26C081FF04C083
:102DD0006091090184E005C082FF07C0609109018C
:102DE00088E0689FB001112417C090917002992368
:102DF000D1F060910801961788F72091090188E0C9
:102E0000289F90011124929FA001939F500D11249F
:102E100070E0CA010E94CB286038710540F461154A
:102E2000710519F406C068E070E0862F08958FE7F9
:102E3000089581E008958091710280FF08C060913B
:102E4000050170E0759567957595679521C081FFBF
:102E500006C06091050170E07595679519C082FF05
:102E600004C06091050170E010C090916F02992339
:102E700099F0609104019617A0F780910501899F50
:102E8000C001112470E00E94CB286038710540F425
:102E90006115710519F406C061E070E0862F089590
:102EA0008FE7089581E008958D3E21F40E94DC169D
:102EB000819504C08E3E29F40E94DC168093750231
:102EC00008958F3E21F40E94DC16819504C0803F56
:102ED00029F40E94DC16809374020895893F19F446
:102EE0000E941B1705C08A3F31F40E941B17819571
:102EF0008093760208958B3F21F40E941B178195E1
:102F000004C08C3F29F40E941B1780937702089518
:102F10009FE0980F983078F421E030E0A90102C0DA
:102F2000440F551F9A95E2F7CA0190917302892BBD
:102F30008093730208958D3F21F480917102816026
:102F40000BC08E3F21F480917102826005C08F3FDB
:102F500029F48091710284608093710208958D3EFE
:102F600039F49091750297FF35C01092750259C0DF
:102F70008E3E29F4909175021916BCF32BC09091E6
:102F800074028F3E29F497FF25C01092740249C045
:102F9000803F19F41916CCF31DC090917602893F39
:102FA00029F41916BCF4109276023BC08A3F19F43A
:102FB00097FF10C0F8CF8B3F39F49091770297FFBD
:102FC00009C0109277022DC08C3F21F490917702B6
:102FD0001916BCF39FE0980F983080F421E030E0A0
:102FE000A90102C0440F551F9A95E2F7CA018095C6
:102FF0009091730289238093730213C08D3F21F453
:10300000809171028E7F0BC08E3F21F480917102FE
:103010008D7F05C08F3F29F4809171028B7F809353
:10302000710280917402811106C080917502811134
:1030300002C01092700280917602811106C08091C8
:103040007702811102C010926F0208958091670289
:1030500083FF7EC087E991E00E9419058091730289
:103060001F928F9382E991E09F938F930E94B20504
:1030700080E991E00E94190580917402282F082EA2
:10308000000C330B3F938F938DE891E09F938F93C8
:103090000E94B2058BE891E00E94190580917502AB
:1030A000282F082E000C330B3F938F9388E891E074
:1030B0009F938F930E94B20586E891E00E941905C4
:1030C00080917602282F082E000C330B3F938F93AC
:1030D00083E891E09F938F930E94B20581E891E08D
:1030E0000E94190580917702282F082E000C330BBF
:1030F0003F938F938EE791E09F938F930E94B20549
:103100008BE791E00E941905809170021F928F93C6
:1031100088E791E09F938F930E94B20586E791E044
:103120000E941905809171021F928F9383E791E0AD
:103130009F938F930E94B20580E791E00E9419054A
:103140008DB79EB74C960FB6F8949EBF0FBE8DBF3D
:103150000E94D82020917402211104C02091750290
:10316000222321F090936E0280936D0220917602CB
:10317000211104C020917702222321F090936C0248
:1031800080936B0282E792E00C94B61FEF92FF925D
:103190000F931F93CF93DF9300D000D000D0CDB713
:1031A000DEB786E0E2E7F2E0DE01119601900D92D3
:1031B0008A95E1F7E0907402F09075020091760232
:1031C000109177021092740210927502109276029A
:1031D00010927702E11003C0FF2009F45DC08091D6
:1031E0006D0290916E020E94F020AC0190917002ED
:1031F000992339F020910A0130E02417350758F05F
:103200004BC020910B018AE0289F900111242417C4
:10321000350718F041C09F3F19F09F5F90937002EF
:10322000EE2061F00E94DC161E1414F09FEF01C026
:1032300091E0989F902D112490937402FF2061F0EB
:103240000E94DC161F1414F09FEF01C091E0989FBC
:10325000902D112490937502309174023323E1F084
:10326000209175022223C1F045EB3403C0011124E3
:10327000992319F09093740203C081E08093740243
:1032800035EB2303C0011124992319F090937502A3
:1032900003C081E080937502011103C0112309F47A
:1032A0005DC080916B0290916C020E94F020AC0195
:1032B00090916F02992339F02091060130E0241794
:1032C000350758F04BC0209107018AE0289F9001F4
:1032D00011242417350718F041C09F3F19F09F5F54
:1032E00090936F02002361F00E941B17101614F0D8
:1032F0009FEF01C091E0989F902D1124909376024A
:10330000112361F00E941B17111614F09FEF01C0EA
:1033100091E0989F902D112490937702309176023E
:103320003323E1F0209177022223C1F045EB3403EF
:10333000C0011124992319F09093760203C081E013
:103340008093760235EB2303C0011124992319F0F1
:103350009093770203C081E080937702809174029A
:1033600081110BC080917502811107C08091760296
:10337000811103C08091770281110E942618EB828F
:10338000FC820D831E8386E0FE013196A2E7B2E047
:1033900001900D928A95E1F726960FB6F894DEBF5C
:1033A0000FBECDBFDF91CF911F910F91FF90EF9096
:1033B0000895E2E7F2E086E0DF011D928A95E9F7E1
:1033C0001092700210926F02109271020895CF93C2
:1033D000DF93EC01FB018281882309F43CC1C430F6
:1033E000FDE5DF0760F4CB3F9CE5D90788F49E013B
:1033F00022503C452431310508F02EC109C0C236A7
:10340000EDE5DE0729F0C63AFDE5DF0709F024C146
:103410000E94811190939B0280939A02C1318CE5A6
:10342000D80709F4C6C008F042C0C930ECE5DE0791
:1034300009F49BC000F5C5308CE5D80709F485C0B8
:1034400078F4C330ECE5DE0709F478C008F07AC000
:10345000C230DC4509F0F5C080919A028160EFC06E
:10346000C7309CE5D90709F478C008F07AC080918C
:103470009A028061E4C0CD30FCE5DF0709F487C023
:1034800058F4CB309CE5D90709F479C008F07BC02B
:1034900080919A0288606FC0CF30FCE5DF0709F4A5
:1034A00080C008F082C080919A02877FC8C0CE3F5A
:1034B0009CE5D90709F471C000F5C531FCE5DF07CB
:1034C00009F485C068F4C3319CE5D90709F475C0D7
:1034D00008F095C00E94200B80919A028F77AFC0B0
:1034E000CC3FFCE5DF07A9F108F054C0CB3FDC4539
:1034F00009F0A7C080919B0240C0C230EDE5DE0715
:1035000009F489C058F4C1158DE5D80709F45AC0EB
:1035100008F069C080919B0282602FC0C236EDE541
:10352000DE0709F47CC0C63AFDE5DF0709F481C077
:10353000C330DD4509F085C080E06EC080919A02FD
:1035400082607DC080919A0216C080919A02886044
:1035500076C080919B0282604FC080919A02806207
:103560006EC080919A0280646AC00E94200B809194
:103570009A02806864C0846062C081603DC08091AE
:103580009A028E7F5CC080919A028D7F58C0809194
:103590009A0216C080919B0218C080919B028D7F79
:1035A0002BC080919A028F7E4AC080919A028F7DB3
:1035B00046C080919A028F7B42C080919A02877F99
:1035C0008B7F3DC080919B028D7F8E7F15C0809147
:1035D0009A0282FB222720F991E0922790FB82F940
:1035E00090FB83F92CC080919B02982F909591704D
:1035F0008E7F892B90FB81F980939B0222C00E94D1
:10360000200B80919A0287FB222720F991E09227D4
:1036100090FB87F914C081E00E94181212C08091BB
:103620009A0284FB222720F991E0922790FB84F9EB
:1036300006C080919A02982F909590FB80F9809314
:103640009A0280919A0290919B020E9492110E948C
:10365000200B80E001C081E0DF91CF91089580913F
:1036600004011F928F93809105011F928F93809187
:1036700008011F928F93809109011F928F9380916F
:103680000A011F928F9380910B011F928F938AEBF7
:1036900091E09F938F930E94B2058DB79EB70E96CF
:1036A0000FB6F8949EBF0FBE8DBF0895883220F5E7
:1036B0008E3108F068C08B3091F1C0F4873009F08A
:1036C000BEC081E080930B0184E180930A018AE00F
:1036D000809309018EE18093080188E080930501C1
:1036E00088E2809304018CE193E0C6C0833109F441
:1036F00043C0843169F1A3C08F3409F49EC028F41B
:10370000893231F1883359F09AC0813531F008F4AB
:10371000D4C0823509F4A7C092C08FEFA5C08EE354
:1037200093E00E9419050E942F1B1F9281E08F9346
:103730001F9288E08F9387E392E09F938F930E947C
:10374000B2050F900F900F900F900F900F9096C0B2
:103750008BE393E00E94190580917C02882309F491
:10376000AAC010927C0210927B0210927A021092F0
:10377000790210927802B1C08DE293E00E9419059F
:103780000E942F1B7BC08D5180937C02833031F1CE
:1037900070F48130D1F0823009F03FC08AE091E0CE
:1037A00090937B0280937A0282E991E01FC085307A
:1037B00059F108F1863089F584E091E090937B021D
:1037C00080937A028DEC91E011C08BE091E09093B0
:1037D0007B0280937A0289E891E008C089E091E059
:1037E00090937B0280937A028EE991E09093790224
:1037F0008093780218C088E091E090937B028093D8
:103800007A028BEA91E0F2CF85E091E090937B021F
:1038100080937A028AEB91E0E9CF10927C028AE2EF
:1038200093E00E94190580917C02882309F455C019
:103830001F928F9386E293E00DC08AE015C089E164
:1038400093E01AC097FF47C0108280811F928F9328
:1038500083E193E09F938F930E94B2050F900F90A6
:103860000F900F900BC081E0E0917A02F0917B0203
:10387000309729F580E193E00E94190520917C02A0
:10388000222359F18091780290917902009711F4E6
:1038900085E891E09F938F931F922F9387E093E0A9
:1038A0009F938F930E94B2050F900F900F900F90EF
:1038B0000F900F9016C080E0089586EFD5CF20813D
:1038C000082E000C990B820F911D8F3F910509F076
:1038D0000CF4B8CF8FEF8083B8CF83E093E00E94E1
:1038E000190581E00895CF93C82F1F928F9384E527
:1038F00093E09F938F930E94B20581E090E0A0E057
:10390000B0E0BC01CD0104C0660F771F881F991F6E
:10391000CA95D2F70E94780B0F900F900F900F90DE
:10392000CF910C94200BEF92FF920F931F93CF93A4
:10393000DF938B3109F4EDC008F08EC08B3009F4B1
:10394000B1C008F078C0863009F4AFC020F48530EB
:1039500009F4BDC04EC1873009F4C0C0883009F0F9
:1039600048C10E947D111F928F9388E797E09F9333
:103970008F930E94B2050E94791183FB992790F9D9
:103980001F929F9382FB992790F91F929F9381FB2F
:10399000992790F91F929F93982F91701F929F9350
:1039A0001F928F938FE297E09F938F930E94B205AF
:1039B0000E94811187FB222720F91F922F9386FBFB
:1039C000222720F91F922F9385FB222720F91F928F
:1039D0002F9384FB222720F91F922F9383FB22270A
:1039E00020F91F922F9382FB222720F91F922F93F9
:1039F00091FB222720F91F922F93292F21701F92CC
:103A00002F9381FB222720F91F922F93282F2170BB
:103A10001F922F939F938F938AE496E09F938F93A7
:103A20000E94B2058DB79EB788960FB6F8949EBFD8
:103A30000FBE8DBF35C0803109F495C020F48E30A3
:103A400009F47BC0D6C0863109F4A8C0893109F0D9
:103A5000D0C084EC93E084C08A32E1F060F4873215
:103A600009F4C3C028F48E3108F4C3C08D51BEC020
:103A7000893269F1BEC0833448F48A3308F0B3C098
:103A8000853309F4B2C0883369F0B3C0833409F4D4
:103A9000ACC0AFC083E298E00E9419050E941612E4
:103AA000C1E0ACC087EA94E05BC080916702817F8F
:103AB0008E7F8093670280E894E00E9419058FE171
:103AC00098E00E94190581E080937D02E9CF83E0B0
:103AD00098E00E9419050E941206E2CF80916702C9
:103AE000C82FC095C170C0FB80F980936702CC23BA
:103AF00029F087EF97E00E94190580C08AEE97E0D1
:103B00000E94190580916702897F877F80936702F1
:103B1000C7CF9091670291FBCC27C0F981E0C827FD
:103B2000892FC0FB81F980936702CC2319F08DEDBA
:103B300097E029C08FEC97E013C09091670292FB49
:103B4000CC27C0F981E0C827892FC0FB82F9809378
:103B50006702CC2319F080EC97E015C080EB97E06A
:103B60000E9419059DCF9091670293FBCC27C0F965
:103B700081E0C827892FC0FB83F980936702CC239B
:103B800051F084EA97E00E941905809167028160F4
:103B90008093670233C087E997E0E2CF0E94E42078
:103BA000162F072FF82EE92ED0919902C0911801F7
:103BB0000E94611FEF92FF920F931F931F92DF935A
:103BC0001F92CF931F928F9389E593E09F938F93DA
:103BD0000E94B2058DB79EB70C960FB6F8949EBFA3
:103BE0000FBE8DBF5DCF895301C080E00E94731C62
:103BF00057CF85E997E00E941905C0E08C2FDF912F
:103C0000CF911F910F91FF90EF90089580E008955C
:103C10000C94061ECF93C82F80917D02813071F0E5
:103C200040F0823009F045C08C2F0E94561B81E085
:103C300046C00E9471108232F1F504C00E947110DA
:103C4000823261F48C2F0E94081E811104C08C2FD7
:103C50000E94931C2CC081E090E029C08C2F0E9410
:103C6000061E811123C0C431C9F058F4CB3069F06D
:103C7000C031B9F482E080937D0288E30E94561B34
:103C800015C0C93259F0C83361F480E894E00E944D
:103C9000190580E593E00E94190508C010927D0285
:103CA0000CC08EE493E00E94190507C081E081708A
:103CB00006C010927D0280E002C080E0F8CFCF9174
:103CC0000895CF93DF9386319C4541F5EB010E9427
:103CD0007110982F8A81209102013091030188236D
:103CE00079F09A7A81E009F480E080937E02911164
:103CF00002C069E201C065E3C9010E9432200AC026
:103D000080917E02811102C069E201C065E3C901B0
:103D10000E9434200E94B31080E001C081E0DF9156
:103D2000CF9108950F931F93CF93DF93C42FD22F7A
:103D3000FC0182818823C9F0409381020E94D8202F
:103D40009093800280937F0280E28C0F883008F08D
:103D500057C0C77081E001C0880FCA95EAF7DF91AC
:103D6000CF911F910F910C947D088091810248138F
:103D700030C080917F02909180020E94F020883CA8
:103D8000910538F510E21D0FCD17B9F080E28C0FC8
:103D9000883040F4C77081E001C0880FCA95EAF707
:103DA0000E948408183028F581E09D2F977001C08B
:103DB000880F9A95EAF70E947D08802F0E94740868
:103DC0001830F0F4D77081E001C0880FDA95EAF777
:103DD0000AC080E28C0F883098F4C77081E001C07F
:103DE000880FCA95EAF7DF91CF911F910F910C943C
:103DF0008408802FDF91CF911F910F910C9474084C
:103E0000DF91CF911F910F9108950F939C01CB01EA
:103E1000243F4CE5340731F188F4293DFCE53F07A8
:103E2000D9F02A3D4CE5340779F1283D3C45A9F508
:103E300006E221EE41EE68ED7CE52BC0263FFCE575
:103E40003F07E1F0A8F0273F3C4539F507E225EEB2
:103E500046EE67EF7CE51DC007E225EE45EE69ED15
:103E60007CE517C006E221EE40EE64EF7CE511C070
:103E700007E225EE44EE65EF7CE50BC006E221EE9D
:103E800042EE66EF7CE505C008E221E045EE6AED12
:103E90007CE50E94921E80E008C0FC01828188239C
:103EA00019F01092810201C081E00F910895909362
:103EB000F3018093F2010895909387028093860224
:103EC0000895E0918602F0918702309721F00190E9
:103ED000F081E02D099480E00895EF92FF920F9316
:103EE0001F93CF93DF93E0918602F0918702309782
:103EF000B1F18C010280F381E02D09958091670278
:103F000082FF2DC080FF04C08CE398E00E94190559
:103F1000E80118E086E3E82E88E0F82E8091670239
:103F200080FF0BC088811F928F93FF92EF920E94B7
:103F3000B2050F900F900F900F9011502196111114
:103F4000EDCF8091670280FF0AC084E398E0DF91A3
:103F5000CF911F910F91FF90EF900C941905DF9175
:103F6000CF911F910F91FF90EF900895E0918602FD
:103F7000F0918702309739F022E0DC012C93048025
:103F8000F581E02D099408952091840230918502F5
:103F90002817390771F09093850280938402E0918D
:103FA0008602F0918702309721F00680F781E02D9C
:103FB00009940895209182023091830228173907CD
:103FC00071F09093830280938202E0918602F091D7
:103FD0008702309721F00084F185E02D099408953F
:103FE000FC01329697E080E0915029F02191222344
:103FF000D9F38F5FF9CF0895662349F0FC0132961B
:1040000008962191621729F0E817F907D1F780E0A7
:10401000089581E008959C01FC0132969FEF80E0B5
:104020004191461789F09F3F19F4411101C0982F23
:104030008F5F8630A9F79F3F39F0F901E90FF11D35
:1040400097FDFA956283089508959C012A5F3F4F7A
:10405000FC014281461301C0128201968217930728
:10406000B9F708950C940B200C942520029626E0B5
:10407000FC0111922A95E9F7089508950C943D20CA
:1040800083E0809388020C943E20811102C081E07D
:1040900001C082E0809388020C943E200C9445205D
:1040A00081E0809388020C943E200C945020089567
:1040B0000C9457200C9458200C9457200C945720A3
:1040C0000C945720CF930E945E200E943E160E94BF
:1040D0005C20C0E08C2F0E942C15811104C0CF5FA2
:1040E000C630C1F701C081E0CF91089508951F92B5
:1040F0000F920FB60F9211248F939F93AF93BF939C
:1041000080918902811113C08091A8029091A90227
:10411000A091AA02B091AB024196A11DB11D80935E
:10412000A8029093A902A093AA02B093AB02BF91F8
:10413000AF919F918F910F900FBE0F901F90189588
:104140008091B002843031F10E949206109289026F
:1041500020E488E190E00FB6F894A8958093600081
:104160000FBE2093600083B7817F846083BF83B7D5
:10417000816083BF7894889583B78E7F83BF0FB6A5
:10418000F894A895809160008861809360001092F7
:1041900060000FBE08950E94200B0C94960682E0EA
:1041A00084BD93E095BD9AEF97BD80936E0008950E
:1041B0002FB7F8948091A8029091A902A091AA0229
:1041C000B091AB022FBF08952FB7F8946091A80269
:1041D0007091A9028091AA029091AB022FBF08951D
:1041E0009C014FB7F8948091A8029091A902A091E8
:1041F000AA02B091AB024FBF821B930B0895789433
:104200001F920F920FB60F9211248F939F93AF932B
:10421000BF938091A8029091A902A091AA02B091A7
:10422000AB020196A11DB11D8093A8029093A90233
:10423000A093AA02B093AB02BF91AF919F918F91CF
:104240000F900FBE0F901F90189587E797E79093F8
:104250000108809300089AE088E10FB6F894A895C9
:10426000809360000FBE90936000FFCF8091980212
:104270000895089522E02093E9002FEF3091E8009F
:10428000215035FD06C035ED3A95F1F700002111BA
:10429000F5CF2091E80025FF0BC040E050E066E03C
:1042A00070E00E9422248091E8008E778093E800DD
:1042B0000895CF93DF9321E02093E9002FEF309111
:1042C000E800215035FD06C035ED3A95F1F70000C4
:1042D0002111F5CF2091E80025FF14C0EC0140E04A
:1042E00050E068E070E00E9422248091E8008E7720
:1042F0008093E80088E0FE01A0E9B2E001900D9211
:104300008A95E1F7DF91CF91089580938C027093A5
:104310008E0260938D028091B002843001F582E0BC
:104320008093E9008FEF9091E800815095FD06C0E1
:1043300095ED9A95F1F700008111F5CF8091E80095
:1043400085FF0DC040E050E063E070E08CE892E053
:104350000E9422248091E8008E778093E8000895DF
:10436000BC0184E00C948521BC0183E00C94852180
:1043700082E698E00E9419058091AF02811109C080
:104380000E94B3250E9410268091E20084608093F1
:10439000E20008958EE598E00E9419051092AF02A0
:1043A00008958AE598E00E9419050C94552086E549
:1043B00098E00E9419056091AC0281E0611101C092
:1043C00080E00C94402082E598E00E9419059091CD
:1043D000B00281E0943009F080E06091AC020C946E
:1043E000452020918B022F5F822F62E30E94BF281D
:1043F000992319F020938B02089510928B028091DB
:104400008F02882371F18091B002843041F5809150
:10441000E9008F702091EC00922F917020FD90E8C0
:10442000892B93E09093E9009091EB0090FF14C0EA
:104430009091EE0097FF10C09091E80095FF03C0A7
:104440001092F100F9CF9091E80090FF05C0909193
:10445000E8009E779093E8008F708093E9001092B7
:104460008F02089542E061EC81E00E942C2542E237
:1044700061EC82E00E942C2542E261EC83E00E9424
:104480002C259091B00281E0943009F080E0609199
:10449000AC020C944E208091B202833009F461C0CA
:1044A00030F4813071F0823009F49AC008958A3076
:1044B00009F486C08B3009F46CC0893009F0A8C0BB
:1044C00020C08091B102813A09F0A2C08091E80039
:1044D000877F8093E8008091B5029091B602892B86
:1044E00021F468E080E992E003C060E080E090E0C1
:1044F00070E00E946D248091E8008B778093E80043
:1045000008958091B102813209F082C08091B50294
:104510009091B602029708F07BC08091E800877FF7
:104520008093E8008091E80082FD05C08091B00290
:104530008111F8CF6DC02091F3008091F20090E0DE
:10454000922B029731F48091F100813011F0863086
:1045500021F48091F100809398028091E8008B779C
:1045600053C08091B102813A09F052C08091B502E6
:104570009091B602892B09F04BC08091E800877FAB
:104580008093E8008091E80080FFFCCF80911801C3
:1045900036C08091B1028132D9F58091B5029091F7
:1045A000B602892BA9F58091E800877F8093E80007
:1045B0000E9461258091B302809318010C94200B16
:1045C0008091B102813221F58091E800877F80934C
:1045D000E8000E9461258091B402809399020895B9
:1045E0008091B102813AA1F48091E800877F8093A5
:1045F000E8008091E80080FFFCCF809199028093D1
:10460000F1008091E8008E778093E8000C9461259A
:1046100008959FB7F89410928F029FBF9091B002B7
:10462000943009F057C09091E9009F703091EC00F0
:10463000232F217030FD20E8922B23E02093E90006
:104640002091EB0020FF43C02091EE0027FF3FC0E8
:1046500020918A02222321F02091E80025FF37C013
:1046600010928A0226E03091E80035FD15C03091A5
:10467000B002343061F53091EB0035FD28C0215097
:1046800021F481E080938A0222C0EFE9FFE03197B4
:10469000F1F700C00000E7CF8093F1008091E800BF
:1046A00085FD0AC08091E80080FFFCCF8091E80082
:1046B0008E778093E80006C08FB7F89421E02093AE
:1046C0008F028FBF9F709093E90080E008959F70E4
:1046D0009093E9008FEF089584B7877F84BF0FB66A
:1046E000F894A89580916000886180936000109292
:1046F00060000FBE90E080E80FB6F89480936100F0
:10470000909361000FBE0C9450200E94B3250E942C
:104710001026E2EEF0E080818460808378940C942F
:10472000A4288CE091E00C945C1F8091B00285304D
:10473000C9F48EE498E00E9419058091B00285309A
:1047400079F40E94A0208091AE028823B1F30E94E8
:104750006220882391F30E940C240E94200BEDCF4D
:104760000C94CB20089508950C94B623292F332759
:1047700023303105C9F060F42130310581F0223059
:10478000310509F041C08BE590E022E938E040C0F6
:1047900021323105E1F02232310531F135C082E1BB
:1047A00090E02DEE38E034C099278130910549F032
:1047B00028F0029749F5E6E6F8E005C0EEE8F8E0F3
:1047C00002C0E8E7F8E0849190E09F0121C06330E7
:1047D0007105D0F4660F771FFB01E551FE4F208174
:1047E000318189E090E014C06330710568F4FB0109
:1047F000EE0FFF1FEB51FE4F20813181FB01EE5187
:10480000FE4F808190E004C080E090E020E030E046
:10481000FA0131832083089580E189BD82E189BD59
:1048200009B400FEFDCF8091D8008F7D8093D80021
:104830008091E00082608093E0008091E00081FD43
:10484000FCCF0895CF92DF92EF92FF920F931F93C8
:10485000CF93DF93EC018B017A010E9480258111B7
:1048600033C0E114F10439F0F70180819181081B14
:10487000190BC80FD91FC12CD12C0115110519F125
:104880008091E80085FD16C08091E8008E778093C6
:10489000E800E114F10449F0F70180819181C80E2C
:1048A000D91ED182C08285E00FC00E948025882356
:1048B00021F30AC089918093F10001501109FFEFA3
:1048C000CF1ADF0ADACF80E0DF91CF911F910F91ED
:1048D000FF90EF90DF90CF9008952091B702309134
:1048E000B8022617370748F06115710539F4209191
:1048F000E8002E772093E80001C0B901FC0120E018
:104900006115710579F18091B0028823F1F185304C
:10491000F1F18091E80083FD3CC08091E80082FDC8
:104920002EC08091E80080FFEBCF2091F3008091B2
:10493000F20090E0922B6115710551F088309105DD
:1049400038F421912093F100615071090196F3CF61
:1049500021E0089709F020E08091E8008E778093AD
:10496000E800CECF2111CFCF0AC08091B0028823BA
:1049700061F0853061F08091E80083FD0AC080918C
:10498000E80082FFF2CF80E0089582E0089583E09E
:10499000089581E008952091B7023091B80226175A
:1049A000370748F06115710539F42091E8002E773A
:1049B0002093E80001C0B901FC0120E061157105F8
:1049C00091F18091B002882309F440C0853009F448
:1049D0003FC08091E80083FD3DC08091E80082FDEA
:1049E0002FC08091E80080FFE9CF2091F3008091F3
:1049F000F20090E0922B6115710559F08830910515
:104A000040F424912093F100319661507109019690
:104A1000F2CF21E0089709F020E08091E8008E773E
:104A20008093E800CBCF2111CCCF0AC08091B00297
:104A3000882361F0853061F08091E80083FD0AC031
:104A40008091E80082FFF2CF80E0089582E008952F
:104A500083E0089581E00895982F973068F590934A
:104A6000E900981739F07091EC002091ED00509119
:104A7000F00003C0242F762F50E021FD02C09F5F7D
:104A8000ECCF3091EB003E7F3093EB003091ED00A6
:104A90003D7F3093ED003091EB0031603093EB00BF
:104AA0007093EC002093ED005093F0002091EE0005
:104AB00027FDE5CF80E008958F708093E90081E0C5
:104AC00008958091B10287FF11C08091E80082FDB6
:104AD00005C08091B0028111F8CF11C08091E8002B
:104AE0008B770BC08091B002882349F08091E80059
:104AF00080FFF8CF8091E8008E778093E8000895DA
:104B00002091E4003091E50095E64091EC00842F7F
:104B1000817040FF23C08091E80080FD1DC080911E
:104B2000B002882399F0853099F08091EB0085FDE3
:104B300011C04091E4005091E5002417350729F396
:104B4000915011F09A01E1CF84E0089582E0089538
:104B500083E0089581E0089580E008954091E800A1
:104B600042FFDDCF08950E9421260E942926E0EE13
:104B7000F0E0808181608083E8EDF0E080818F77D4
:104B8000808319BCA7EDB0E08C918E7F8C938081DF
:104B90008F7E80831092AF0208950F931F93CF935F
:104BA000DF930E9421260E942926C8EDD0E088814B
:104BB0008F77888388818068888388818F7D8883C8
:104BC00019BC1092B0021092AC021092AE02109278
:104BD000AD0200EE10E0F80180818B7F8083888138
:104BE0008160888342E060E080E00E942C25E1EE55
:104BF000F0E080818E7F8083E2EEF0E08081816052
:104C00008083808188608083F80180818E7F8083AB
:104C1000888180618883DF91CF911F910F910895E2
:104C2000E8EDF0E080818F7E8083E7EDF0E0808129
:104C30008160808384E082BF81E08093AF020C9426
:104C4000CD25E8EDF0E080818E7F80831092E20038
:104C500008951092DA001092E10008951F920F92C9
:104C60000FB60F9211242F933F934F935F936F933F
:104C70007F938F939F93AF93BF93EF93FF93809115
:104C8000E10082FF0BC08091E20082FF07C08091AB
:104C9000E1008B7F8093E1000E94F1218091DA0096
:104CA00080FF1FC08091D80080FF1BC08091DA0078
:104CB0008E7F8093DA008091D90080FF0DC080E163
:104CC00089BD82E189BD09B400FEFDCF81E08093FA
:104CD000B0020E94B82105C019BC1092B0020E9417
:104CE000CA218091E10080FF19C08091E20080FF1D
:104CF00015C08091E2008E7F8093E2008091E200F7
:104D000080618093E2008091D80080628093D80017
:104D100019BC85E08093B0020E94D7218091E10008
:104D200084FF30C08091E20084FF2CC080E189BD07
:104D300082E189BD09B400FEFDCF8091D8008F7D4E
:104D40008093D8008091E1008F7E8093E100809174
:104D5000E2008F7E8093E2008091E2008160809388
:104D6000E2008091AC02882311F084E007C08091BA
:104D7000E30087FD02C081E001C083E08093B002C0
:104D80000E94E3218091E10083FF29C08091E2002D
:104D900083FF25C08091E100877F8093E10082E05E
:104DA0008093B0021092AC028091E1008E7F8093DC
:104DB000E1008091E2008E7F8093E2008091E2002A
:104DC00080618093E20042E060E080E00E942C2558
:104DD0008091F00088608093F0000E94D121FF91C3
:104DE000EF91BF91AF919F918F917F916F915F9163
:104DF0004F913F912F910F900FBE0F901F901895DC
:104E00001F920F920FB60F9211242F933F934F933F
:104E10005F936F937F938F939F93AF93BF93CF9342
:104E2000DF93EF93FF93C091E900CF708091EC0086
:104E3000D82FD17080FDD0E81092E9008091F00069
:104E4000877F8093F00078940E9444271092E900B5
:104E50008091F00088608093F000CD2BCF70C093DC
:104E6000E900FF91EF91DF91CF91BF91AF919F91B9
:104E70008F917F916F915F914F913F912F910F9003
:104E80000FBE0F901F9018951F93CF93DF93CDB750
:104E9000DEB7AA970FB6F894DEBF0FBECDBFE1EB29
:104EA000F2E08091F100819322E0E93BF207C9F73B
:104EB0000E944B228091E80083FF2EC18091B102B5
:104EC0009091B202492F50E04A30510508F024C1B8
:104ED000FA01EE59FF4F0C94DF28803821F0823818
:104EE00009F01AC108C08091AD029091AE029923D9
:104EF00089F082600FC08091B5028F70873008F012
:104F00000BC18093E9008091EB0085FB882780F935
:104F10001092E9009091E800977F9093E8008093C9
:104F2000F1001092F100D1C0282F2D7F09F0F4C0BC
:104F3000882319F0823061F0EFC08091B302813094
:104F400009F0EAC0933009F080E08093AE022EC0F1
:104F50008091B30281112AC08091B5028F702FEF2A
:104F6000280F263008F0D8C08093E9002091EB008C
:104F700020FF1CC0933021F48091EB00806214C0AC
:104F80009091EB0090619093EB0021E030E0A9015B
:104F900002C0440F551F8A95E2F74093EA00109231
:104FA000EA008091EB0088608093EB001092E900AA
:104FB0008091E800877F8093E8000E946125ACC063
:104FC0008111AAC01091B3021F778091E30080780D
:104FD000812B8093E3008091E800877F8093E80035
:104FE0000E9461258091E80080FFFCCF8091E30062
:104FF00080688093E300111102C082E001C083E069
:105000008093B00289C08058823008F085C08091BA
:10501000B3029091B4028C3D53E0950779F583E09B
:105020008A838AE289834FB7F894DE01139620E0E1
:105030003EE051E2E32FF0E050935700E49120FF6F
:1050400003C0E295EF703F5FEF708E2F90E0EA3083
:1050500010F0C79601C0C0968D939D932F5F2431A9
:1050600049F74FBF8091E800877F8093E8006AE2AC
:1050700070E0CE0101960E946D2416C06091B502C9
:105080007091B602AE014F5F5F4F0E94B423BC0126
:10509000892B09F441C09091E800977F9093E80034
:1050A00089819A810E94CB248091E8008B7780933C
:1050B000E80032C0803881F58091E800877F8093D6
:1050C000E8008091AC028093F1008091E8008E7737
:1050D00072CF811121C08091B3029091B4029927BF
:1050E0000297D4F48091E800877F8093E800809154
:1050F000B3028093AC020E9461258091AC028111C1
:1051000006C08091E30087FD02C081E001C084E019
:105110008093B0020E9432228091E80083FF0AC08F
:105120008091E800877F8093E8008091EB008062A7
:105130008093EB00AA960FB6F894DEBF0FBECDBFEA
:10514000DF91CF911F910895CF938091B002882372
:10515000A1F0C091E900CF709091EC00892F81708F
:1051600090FD80E8C82B1092E9008091E80083FD53
:105170000E944427CF70C093E900CF910895991BF6
:1051800079E004C0991F961708F0961B881F7A953E
:10519000C9F78095089597FB072E16F4009407D061
:1051A00077FD09D00E94E52807FC05D03EF49095D4
:1051B00081959F4F0895709561957F4F0895EE0FEB
:1051C000FF1F0590F491E02D0994AA1BBB1B51E130
:1051D00007C0AA1FBB1FA617B70710F0A61BB70B67
:1051E000881F991F5A95A9F780959095BC01CD010C
:1051F0000895FB01DC0104C08D910190801921F418
:1052000041505040C8F7881B990B0895F999FECF7B
:1052100092BD81BDF89A992780B50895A8E1B0E0C4
:1052200042E050E00C943A29262FF999FECF92BD26
:1052300081BDF89A019700B4021639F01FBA20BD5B
:105240000FB6F894FA9AF99A0FBE08950396272F8D
:105250000E9415290E941429252F0E941529242F08
:105260000C9415290196272F0E9415290C941429B6
:10527000DC01CB01FC01F999FECF06C0F2BDE1BD16
:10528000F89A319600B40D9241505040B8F7089505
:04529000F894FFCFC0
:10529400C8004F02280850011E0A14013621592162
:1052A4003A21B421B021392101E200E900EA00B534
:1052B40000B600B700CD008301CC008A01920194AE
:1052C400012102230224022502260227022A02B314
:1052D40000B4006F007000818283E200E900EA00FC
:1052E400B500B600B700CD008301CC008A0192015D
:1052F40094012102230224022502260227022A0203
:10530400B300B4006F00700081828390919293F493
:10531400F5F6F731333F3F3F006D6B5F64656C61B9
:1053240079006D6B5F696E74657276616C006D6B8C
:105334005F6D61785F7370656564006D6B5F746940
:105344006D655F746F5F6D6178006D6B5F77686525
:10535400656C5F6D61785F7370656564006D6B5F2C
:10536400776865656C5F74696D655F746F5F6D61A7
:105374007800407B229C092109FF08A408BD08D6B7
:0253840008001F
:00000001FF
